:100000000C945A000C9477000C9477000C947700B1
:100010000C9477000C9477000C9477000C94770084
:100020000C9477000C9477000C9477000C94770074
:100030000C9477000C9477000C9477000C94770064
:100040000C943E030C9477000C9477000C9477008A
:100050000C9477000C9477000C9477000C94770044
:100060000C9477000C947700000024272A000025C8
:10007000282B000023262904040404040404040299
:100080000202020202030303030303010204081035
:100090002040800102040810200102040810200002
:1000A0000000070002010000030406000000000039
:1000B0000000000011241FBECFEFD4E0DEBFCDBF93
:1000C00011E0A0E0B1E0E2E7FAE002C005900D9295
:1000D000A231B107D9F711E0A2E1B1E001C01D9250
:1000E000AA31B107E1F70E9437030C9438050C944C
:1000F0000000809100010E947F04892B09F0EAC171
:10010000809102010E947F04892B09F0E3C1809154
:1001100004010E947F04892B09F0DCC18091060153
:100120000E947F04892B09F0D5C16FEF70E08091A8
:100130000E010E940D046EEB70E080910C010E9494
:100140000D046CE870E0C1C1809102010E947F043F
:10015000892B09F0C6C1809104010E947F04892B7C
:1001600009F0BFC1809106010E947F04019709F048
:10017000B8C16FEF70E017C0809102010E947F0448
:10018000892B09F0B5C1809104010E947F04019779
:1001900009F0AEC1809106010E947F04892B09F00D
:1001A000A7C164E670E080910E010E940D046FEF1C
:1001B00070E071C0809102010E947F04892B09F0D8
:1001C0009EC1809104010E947F04019709F097C1AC
:1001D000809106010E947F04019709F090C16FEFA2
:1001E00070E053C0809102010E947F04019709F0E2
:1001F0008DC1809104010E947F04892B09F086C182
:10020000809106010E947F04892B09F07FC16FEF66
:1002100070E017C0809102010E947F04019709F0ED
:100220007CC1809104010E947F04892B09F075C173
:10023000809106010E947F04019709F06EC164E677
:1002400070E080910E010E940D046FEF70E08091CC
:100250000C010E940D0464E670E037C18091020138
:100260000E947F04019709F05FC1809104010E9400
:100270007F04019709F058C1809106010E947F0414
:10028000892B09F051C164E670E080910E010E9453
:100290000D0464E670E080910C010E940D046FEF84
:1002A00070E013C1809102010E947F04019709F060
:1002B00042C1809104010E947F04019709F03BC173
:1002C000809106010E947F04019709F034C16FEF0D
:1002D00070E017C0809102010E947F04892B09F011
:1002E00031C1809104010E947F04892B09F02AC149
:1002F000809106010E947F04892B09F023C164E6E6
:1003000070E080910E010E940D0464E670E09FCFC2
:10031000809102010E947F04892B09F01AC180910B
:1003200004010E947F04892B09F013C1809106010A
:100330000E947F04019709F00CC169E170E080918F
:100340000E010E940D0464EB70E080910C010E948C
:100350000D0468E770E0B9C0809102010E947F043B
:10036000892B09F0FDC0809104010E947F04019750
:1003700009F0F6C0809106010E947F04892B09F0E4
:10038000EFC062E870E080910E010E940D046FEFF3
:1003900070E080910C010E940D0468EC70E095C043
:1003A000809102010E947F04892B09F0E0C08091B6
:1003B00004010E947F04019709F0D9C080910601D1
:1003C0000E947F04019709F0D2C06AEA70E0809130
:1003D0000E010E940D0467E070E05DCF8091020184
:1003E0000E947F04019709F0C9C0809104010E9416
:1003F0007F04892B09F0C2C0809106010E947F040E
:10040000892B09F0BBC060E070E0CDCE8091020185
:100410000E947F04019709F0B8C0809104010E94F6
:100420007F04892B09F0B1C0809106010E947F04EE
:10043000019709F0AAC06FEF70E080910E010E9451
:100440000D0460E070E027CF809102010E947F04DC
:10045000019709F0A1C0809104010E947F040197D7
:1004600009F09AC0809106010E947F04892B09F04F
:1004700093C06FEF70E080910E010E940D046FEF4A
:1004800070E01DC0809102010E947F04019709F075
:100490008AC0809104010E947F04019709F083C003
:1004A000809106010E947F04019709F07CC060E002
:1004B00070E080910E010E940D0460E070E0809178
:1004C0000C010E940D0460E070E080910A010E941E
:1004D0000D040895809100010E947F04892B09F486
:1004E00033CE809100010E947F04892B09F444CE11
:1004F000809100010E947F04892B09F45BCE8091DA
:1005000000010E947F04892B09F46CCE80910001C8
:100510000E947F04892B09F47DCE809100010E9406
:100520007F04892B09F49ACE809100010E947F04F8
:10053000892B09F4B7CE809100010E947F040197B6
:1005400009F4C8CE809100010E947F04019709F44C
:10055000DFCE809100010E947F04019709F4FCCE58
:10056000809100010E947F04019709F419CF8091C6
:1005700000010E947F04019709F430CF80910001AF
:100580000E947F04019709F441CF809100010E94ED
:100590007F04019709F458CF809100010E947F04E5
:1005A000019709F46FCF089560E0809100010E94E7
:1005B000610460E0809102010E94610460E080912A
:1005C00004010E94610460E0809106010E946104C0
:1005D00061E0809108010E94610461E080910E0158
:1005E0000E94610461E080910C010E94610461E05D
:1005F00080910A010E9461046FEF70E080910E010A
:100600000E940D046AE570E080910C010E940D04C7
:1006100062E370E080910A010E940D0460ED77E0D2
:1006200080E090E00E947B0360E070E080910E012A
:100630000E940D0460E070E080910C010E940D04A6
:1006400060E070E080910A010E940D0461E08091F9
:1006500008010E94CB0464E670E080E090E00E9414
:100660007B0360E0809108010E94CB0408950E9402
:10067000AA030E94D4020E947900FDCF1F920F921C
:100680000FB60F9211248F939F93AF93BF938091D6
:10069000160190911701A0911801B09119010196CE
:1006A000A11DB11D8093160190931701A09318010D
:1006B000B0931901BF91AF919F918F910F900FBE91
:1006C0000F901F90189560911601709117018091FD
:1006D00018019091190127E0660F771F881F991F55
:1006E0002A95D1F72DE730E040E050E00E94160552
:1006F000CA01B9010895AF92BF92CF92DF92EF92F3
:10070000FF920F931F935B016C010E9463037B01B7
:100710008C010E9463036E197F09800B910B6A158F
:100720007B058C059D05A8F31F910F91FF90EF901D
:10073000DF90CF90BF90AF900895019751F0880F50
:10074000991F880F991F02972FB7F8940197F1F717
:100750002FBF0895789410921601109217011092ED
:1007600018011092190184B5826084BD84B581603E
:1007700084BD85B5826085BD85B5816085BDEEE6A9
:10078000F0E0808181608083E1E8F0E08081826038
:100790008083808181608083E0E8F0E080818160F7
:1007A0008083E1EBF0E0808184608083E0EBF0E027
:1007B000808181608083EAE7F0E0808184608083CB
:1007C0008081826080838081816080838081806875
:1007D00080831092C1000895809310010895909134
:1007E00010019295990F990F907C8F70982B909390
:1007F0007C0080917A00806480937A0080917A00F6
:1008000086FDFCCF20917800809179009927982F60
:1008100088273327822B932B08951F93CF93DF9341
:10082000182FEB0161E00E946104E12FFF27E156E0
:10083000FF4F8491833051F48091800080688093D1
:100840008000D0938900C093880037C0843051F471
:1008500080918000806280938000D0938B00C09351
:100860008A002BC0813029F484B5806884BDC7BD5F
:1008700024C0823029F484B5806284BDC8BD1DC007
:10088000863041F48091B00080688093B000C093BE
:10089000B30013C0873041F48091B0008062809330
:1008A000B000C093B40009C0C038D10514F460E0B2
:1008B00001C061E0812F0E94CB04DF91CF911F9195
:1008C0000895282F3327C90185579F4FFC01949124
:1008D00029583F4FF9018491882381F0E82FFF27A1
:1008E000E859FF4FE491FF27662329F48081909512
:1008F0008923808308958081892B80830895482FE0
:100900005527CA0181569F4FFC012491CA01855782
:100910009F4FFC01949149585F4FFA013491332362
:1009200019F480E090E00895222331F1233021F47E
:10093000809180008F7705C0243031F48091800051
:100940008F7D8093800018C0213019F484B58F7793
:1009500004C0223021F484B58F7D84BD0DC02630C3
:1009600021F48091B0008F7705C0273029F4809161
:10097000B0008F7D8093B000E32FFF27EE58FF4F2C
:10098000E491FF27808120E030E0892311F021E00D
:1009900030E0C9010895482F5527CA0181569F4F5D
:1009A000FC012491CA0185579F4FFC01949149583D
:1009B0005F4FFA0134913323C1F1222331F1233007
:1009C00021F4809180008F7705C0243031F480912C
:1009D00080008F7D8093800018C0213019F484B589
:1009E0008F7704C0223021F484B58F7D84BD0DC083
:1009F000263021F48091B0008F7705C0273029F48C
:100A00008091B0008F7D8093B000E32FFF27E359E2
:100A1000FF4FE491FF27662329F480819095892375
:100A2000808308958081892B80830895A1E21A2E06
:100A3000AA1BBB1BFD010DC0AA1FBB1FEE1FFF1F82
:100A4000A217B307E407F50720F0A21BB30BE40BD2
:100A5000F50B661F771F881F991F1A9469F7609519
:100A60007095809590959B01AC01BD01CF010895D3
:020A7000FFCFB6
:100A72000200030004000500060009000A000B0042
:020A8200010071
:00000001FF
